:0421000002211B326B
:03210B00022209A4
:0321130002220C99
:0B217400E4F508F509750A00750B0082
:0321820002211621
:052116001225E080FE2F
:20218500C00D85810DAC82AD83AEF0FFE5812408F581E50D2405F8E4F608F608F608F6E58B
:2021A5000D2405F8C3E69C08E69D08E69E08E69F504CA80D08E4F608F608F608F6A80D0819
:2021C500C3E6943208E6940008E6940008E694005015A80D08740126F6E40836F6E4083618
:2021E500F6E40836F680D6E50D2405F8740126F6E40836F6E40836F6E40836F680A1850DD7
:2022050081D00D22050B32C020C0E0C0F0C082C083C007C006C005C004C003C002C001C026
:2022250000C0D075D000C374F4950874818509F063F08095F0E433FF7024E50A7020742074
:20224500C0E09000041226911581750A010508E4B508020509758CFC758A1702258BEF7084
:20226500257401B50A20743CC0E09000041226911581750A000508E4B508020509758CFC63
:20228500758A1702258BEF6035C374B4950874838509F063F08095F04024E50A7020742021
:2022A500C0E09000041226911581750A010508E4B508020509758CFB758A8B02258BEF60C1
:2022C50036C374B4950874838509F063F08095F040257401B50A20743CC0E0900004122699
:2022E500911581750A000508E4B508020509758CFB758A8B02258BC374B495087483850930
:20230500F063F08095F0E433FF6035C3743A950874858509F063F08095F04024E50A702005
:202325007420C0E09000041226911581750A010508E4B508020509758CFA758AFF02258B88
:20234500EF6036C3743A950874858509F063F08095F040257401B50A20743CC0E090000479
:202365001226911581750A000508E4B508020509758CFA758AFF02258BC3743A950874850A
:202385008509F063F08095F0E433FF6035C37497950874868509F063F08095F04024E50A29
:2023A50070207420C0E09000041226911581750A010508E4B508020509758CFA758A6902BE
:2023C500258BEF6036C37497950874868509F063F08095F040257401B50A20743CC0E090EF
:2023E50000041226911581750A000508E4B508020509758CFA758A6902258BC374979508B8
:2024050074868509F063F08095F0E433FF6035C374E0950874878509F063F08095F0402453
:20242500E50A70207420C0E09000041226911581750A010508E4B508020509758CFA758AB9
:202445000F02258BEF6036C374E0950874878509F063F08095F040257401B50A20743CC083
:20246500E09000041226911581750A000508E4B508020509758CFA758A0F02258BC374E075
:20248500950874878509F063F08095F0E433FF6035C37406950874898509F063F08095F071
:2024A5004024E50A70207420C0E09000041226911581750A010508E4B508020509758CF9D5
:2024C500758A5B02258BEF6036C37406950874898509F063F08095F040257401B50A20748C
:2024E5003CC0E09000041226911581750A000508E4B508020509758CF9758A5B02258BC302
:202505007406950874898509F063F08095F0E433FF6034C3740B9508748A8509F063F080F4
:2025250095F04023E50A701F7420C0E09000041226911581750A010508E4B5080205097556
:202545008CF8758A89803FEF6035C3740B9508748A8509F063F08095F040247401B50A1FBD
:20256500743CC0E09000041226911581750A000508E4B508020509758CF8758A898007E4EA
:20258500F508F509F50AD0D0D000D001D002D003D004D005D006D007D083D082D0F0D0E0EB
:2025A500D02032C00D85810DAE82AF837402F00EBE00010FE50D24FBF886040886058D04B9
:2025C5008E828F83ECF0A3AE82AF83E50D24FBF886058E828F83EDF0D00D22758CFC758A65
:2025E500177589017588117D0C7E227F80C005C006C00790200B1225A81581158115817D5F
:20260500097E227F80C005C006C0079020031225A8158115811581D2AFD2A9D2A8850B82DF
:0526250012266D80F893
:03217F00750C00DC
:20262A00C00D85810DE582FF24F850028032AE0C8FF005F07401800225E0D5F0FBFFE50D4F
:20264A0024FDF8E66005EF42068005EFF4FF5206C006C0069000071226911581D0068E0C24
:20266A00D00D22AF82C007C0079000071226911581D0078F0C22E4C0E09000041226911512
:07268A00819000020226A767
:20269100C00D85810DAD84758408E50D24FDF8E6F08D84D00D22AD84758408E0FE8D848E77
:0226B100822283
:06214A00E478FFF6D8FD69
:202128007900E94400601B7A009026B7780075A060E493F2A308B8000205A0D9F4DAF27521
:02214800A0FFF6
:202150007800E84400600A790075A060E4F309D8FC7800E84400600C7900906000E4F0A3CF
:04217000D8FCD9FAC4
:0D211B007581201226B3E5826003022116B3
:0426B300758200220A
:00000001FF
